:1000000019C048C432C031C030C02FC02EC02DC06E
:100010002CC02BC02AC029C028C027C026C025C09C
:1000200055C023C022C021C020C01FC01EC01DC09B
:100030001CC01BC011241FBECFEFD4E0DEBFCDBF5C
:1000400011E0A0E0B1E0E4ECFAE002C005900D920E
:10005000A030B107D9F711E0A0E0B1E001C01D92D6
:10006000AB39B107E1F712D32CC5CACFCF93DF93D9
:10007000CDB7DEB7E5E4F0E081E08083E6E4F0E0D0
:1000800080E28083AEE6B0E0EEE6F0E08081816061
:100090008C931092010110920201109203011092B0
:1000A00004011092060110920701109208011092AB
:1000B000090110920B0110920C0110920D01109287
:1000C0000E0110920F01DF91CF9108951F920F92B0
:1000D0000FB60F9211242F933F934F935F936F931B
:1000E0007F938F939F93AF93BF93EF93FF93CF93A0
:1000F000DF93CDB7DEB7E6E4F0E080E28083809165
:100100001101909112012FEF8F3F920751F04CF0A7
:1001100080911101909112010196909312018093A8
:100120001101809111019091120120E48130920718
:100130000CF042D38091010190910201A091030142
:10014000B09104010196A11DB11D8093010190930E
:100150000201A0930301B0930401809106019091E4
:100160000701A0910801B09109010196A11DB11DDF
:100170008093060190930701A0930801B0930901B1
:1001800080910C0190910D01A0910E01B0910F0191
:100190000196A11DB11D80930C0190930D01A093B8
:1001A0000E01B0930F0180910A01882389F180919B
:1001B0000B01853079F4ABE2B0E0EBE2F0E0808156
:1001C00080648C93ABE2B0E0EBE2F0E090818FE7EB
:1001D00089238C9380910B018A30A9F410920B0132
:1001E00080910A01815080930A01ABE2B0E0EBE21A
:1001F000F0E080818F7B8C93ABE2B0E0EBE2F0E04B
:10020000808180688C9380910B018F5F80930B01BC
:10021000DF91CF91FF91EF91BF91AF919F918F911E
:100220007F916F915F914F913F912F910F900FBEF2
:100230000F901F901895CF93DF93CDB7DEB7109234
:100240000601109207011092080110920901809195
:10025000060190910701A0910801B0910901803732
:1002600021E1920721E0A20720E0B20784F3DF91A9
:10027000CF910895CF93DF93CDB7DEB710920601EB
:100280001092070110920801109209018091060155
:1002900090910701A0910801B0910901883B2BE0E2
:1002A000920720E0A20720E0B20784F3DF91CF910C
:1002B0000895CF93DF93CDB7DEB722970FB6F894AA
:1002C000DEBF0FBECDBF9A83898389819A819C014D
:1002D000442755278091010190910201A0910301CB
:1002E000B091040182179307A407B50774F3109225
:1002F0000101109202011092030110920401229652
:100300000FB6F894DEBF0FBECDBFDF91CF91089539
:10031000CF93DF93CDB7DEB7ABE2B0E0EBE2F0E036
:1003200080818B7F8C9381E190E0C3DFABE2B0E012
:10033000EBE2F0E0808184608C9381E190E0B9DFB2
:10034000DF91CF910895CF93DF93CDB7DEB7ABE2C6
:10035000B0E0EBE2F0E080818B7F8C9381E190E074
:10036000A8DFABE2B0E0EBE2F0E0808184608C9348
:1003700081E390E09EDFDF91CF910895CF93DF93EB
:10038000CDB7DEB722970FB6F894DEBF0FBECDBF54
:100390008A83ABE2B0E0EBE2F0E0808184608C9392
:1003A00080E098E086DFABE2B0E0EBE2F0E0808155
:1003B0008B7F8C938AEF90E07CDFABE2B0E0EBE2E6
:1003C000F0E0808184608C9386E890E072DFA0DFAB
:1003D0009FDF9EDF9DDF9CDF9BDF9ADF99DFB3DF2E
:1003E000B2DFB1DFB0DFAFDFAEDFADDFACDF81E0CA
:1003F00089839A8189818923882311F0A4DF01C030
:1004000087DF8981880F89839A818981892388235D
:1004100011F099DF01C07CDF8981880F89839A817F
:1004200089818923882311F08EDF01C071DF8981E2
:10043000880F89839A8189818923882311F083DF3A
:1004400001C066DF8981880F89839A818981892328
:10045000882311F078DF01C05BDF8981880F8983F1
:100460009A8189818923882311F06DDF01C050DFD3
:100470008981880F89839A8189818923882311F052
:1004800062DF01C045DF8981880F89839A81898174
:100490008923882311F057DF01C03ADF81E0898387
:1004A0009A8189818923882311F44DDF01C030DFCF
:1004B0008981880F89839A8189818923882311F40E
:1004C00042DF01C025DF8981880F89839A81898174
:1004D0008923882311F437DF01C01ADF8981880F4F
:1004E00089839A8189818923882311F42CDF01C0B3
:1004F0000FDF8981880F89839A81898189238823E5
:1005000011F421DF01C004DF8981880F89839A817A
:1005100089818923882311F416DF01C0F9DE8981DE
:10052000880F89839A8189818923882311F40BDFBD
:1005300001C0EEDE8981880F89839A8189818923B0
:10054000882311F400DF01C0E3DEFDDEABE2B0E0A2
:10055000EBE2F0E0808184608C9380E894E0A9DE97
:10056000ABE2B0E0EBE2F0E080818B7F8C9380E146
:1005700091E09FDEABE2B0E0EBE2F0E080818460EE
:100580008C9380E490E095DEABE2B0E0EBE2F0E04B
:1005900080818B7F8C9382E190E08BDEABE2B0E0D8
:1005A000EBE2F0E0808184608C9322960FB6F894A1
:1005B000DEBF0FBECDBFDF91CF910895CF93DF9304
:1005C000CDB7DEB728970FB6F894DEBF0FBECDBF0C
:1005D0001D821C82AC81BD8160D2802DBD83AC8325
:1005E0008E838E8199278F83EFE3F0E080819927B6
:1005F000827090700097C1F7188616C08885992779
:1006000001969A838983A981BA8147D2802DBA83C2
:10061000A9838B838B819927B1DE81E090E011D093
:100620000ADE88858F5F888798858F81981730F3D9
:1006300028960FB6F894DEBF0FBECDBFDF91CF91E5
:100640000895CF93DF93CDB7DEB722970FB6F89416
:10065000DEBF0FBECDBF8A8319820BC088EC8093AA
:100660000A0180910A018823E1F704DE89818F5F06
:10067000898399818A81981788F322960FB6F89416
:10068000DEBF0FBECDBFDF91CF910895CF93DF9333
:10069000CDB7DEB7A4E2B0E0E4E2F0E080818160B3
:1006A0008C93A5E2B0E0E5E2F0E0808181608C937C
:1006B000AAE2B0E0EAE2F0E0808180648C93ABE2F1
:1006C000B0E0EBE2F0E0808180648C93AAE2B0E0DD
:1006D000EAE2F0E0808180688C93ABE2B0E0EBE28C
:1006E000F0E0808180688C93AAE2B0E0EAE2F0E07A
:1006F00080818B7F8C93ABE2B0E0EBE2F0E0808115
:1007000084608C93B3DC69D010920001789482E00D
:1007100098DF8091010190910201A0910301B091B5
:10072000040180342DE0920723E0A20720E0B20705
:1007300084F3809100018823D9F080910C0190917D
:100740000D01A0910E01B0910F01813A2BEB9207A0
:100750002DE0A20720E0B2071CF084E072DFFFCF9B
:1007600080910001853648F385E06BDF64DDFCCFC6
:1007700083E067DF60DDEDE3F0E01082AAE2B0E045
:10078000EAE2F0E0808184608C93ABE2B0E0EBE2DF
:10079000F0E0808184608C9311DFAAE2B0E0EAE2AD
:1007A000F0E080818B7F8C93ABE2B0E0EBE2F0E095
:1007B000808184608C93FFCFCF93DF93CDB7DEB77A
:1007C0008FEF9FEF9093120180931101109210010F
:1007D00010920501DF91CF910895CF93DF93CDB7AC
:1007E000DEB7ADE3B0E0EDE3F0E0808181608C93B3
:1007F000A9E6B0E0E9E6F0E0808181608C93DCDF7F
:10080000DF91CF910895CF93DF93CDB7DEB72997CE
:100810000FB6F894DEBF0FBECDBF888769871092F0
:100820000C0110920D0110920E0110920F0188859B
:100830008F5F1D821C828E838E81AC81BD81082ECC
:1008400034D1BD83AC83EFE3F0E0808199278270DF
:1008500090700097C1F78885992701969A838983BC
:1008600089858B838B81A981BA81082E1ED1BA8399
:10087000A983EFE3F0E08081992782709070009760
:10088000C1F729960FB6F894DEBF0FBECDBFDF913A
:10089000CF9108951F920F920FB60F9211242F93AC
:1008A0003F934F935F936F937F938F939F93AF93F8
:1008B000BF93EF93FF93CF93DF93CDB7DEB7289726
:1008C000DEBFCDBFE9E2F0E08081992784709070AF
:1008D000009761F01092120110921101A5E2B0E0B0
:1008E000E5E2F0E080818E7F8C93C0C080911101A1
:1008F00090911201181619060CF0B1C080911001E8
:10090000282F332738872F838F819885813291054F
:1009100049F12F8138852232310529F08F81988560
:10092000009731F146C0809100019927209105017F
:10093000FC01ED5EFE4F2083809105019091000146
:10094000682F892F60DF809100018F5F8093000105
:10095000809110018F5F809310012EDF8AEF8093CA
:100960000A017EC0809110018F5F8093100178C0D2
:1009700080911101909112011E828C37910514F41F
:1009800091E09E8380911101909112011D82813925
:10099000910514F021E02D838E813D81832B8823E6
:1009A00011F00ADF5DC0809110018F5F809310010C
:1009B00057C080911101909112011C828B309105DA
:1009C00014F481E08C8380911101909112011B82BB
:1009D0008833910514F091E09B838C812B81822BCD
:1009E000882311F0E9DE3CC0809110011A82813128
:1009F00010F031E03A83809110011982893110F4AE
:100A000081E089838A8199818923882311F1A5E274
:100A1000B0E0E5E2F0E0808181608C93809111018B
:100A2000909112018A329105A4F0809110019927CA
:100A30009C012151304081E090E0022E02C0880FDD
:100A4000991F0A94E2F7982F80910501892B8093D2
:100A50000501809110018F5F8093100101C0ACDE11
:100A60008FEF9FEF90931201809311012896F894D5
:100A7000DEBFCDBFDF91CF91FF91EF91BF91AF91DD
:100A80009F918F917F916F915F914F913F912F91A6
:100A90000F900FBE0F901F901895F999FECFB2BD21
:100AA000A1BDF89A119600B40895F999FECFB2BD90
:100AB000A1BD00BC11960FB6F894FA9AF99A0FBE30
:040AC0000895FFCFC7
:00000001FF
